:100000000C94EF030C940C040C940C040C940C044E
:100010000C940C040C940C040C940C040C940C0420
:100020000C940C040C940C040C941F150C94611487
:100030000C94FB1C0C940C040C940C040C940C04F9
:100040000C940C040C940C040C940C040C940C04F0
:100050000C940C040C94AE1C0C940C040C940C0426
:100060000C940C040C940C040C940C040C940C04D0
:100070000C940C040C940C040C940C040C940C04C0
:100080000C940C040C940C040C940C040C940C04B0
:100090000C940C040C940C040C940C040C940C04A0
:1000A0000C940C040C940C040C940C043C06B00648
:1000B00044060E061206480615064B06560620068E
:1000C000A60624065A0628065E0688062C06620640
:1000D000920632066806720619064F061C0652067C
:1000E00037066D067E069E06A0060A064006B9067D
:1000F000E206E806D306D906EE06F406FA0631074C
:1001000057075C07610766076B07700775077A0773
:100110007F0784074408440877087708F60814091D
:10012000150A150A19098D099E099E09CA0ECD0ED8
:10013000000F2D0F340F3F0F420F420F420F901050
:100140009010F90FFB0FFF0F251048104B104E10A9
:10015000711071129812491498124914E41207137D
:100160004914FD130D140000000000000000000001
:10017000000000000000000000000000000000007F
:10018000000000000000000000007E0F00D4FFFF10
:10019000FFC70000007800000000000000002A2BCC
:1001A0002800000000000000000000000000000027
:1001B0000029000000002C1E342021222434262790
:1001C000252E362D3738271E1F20212223242526B1
:1001D0003333362E37381F0405060708090A0B0C7F
:1001E0000D0E0F101112131415161718191A1B1CC7
:1001F0001D2F3130232D350405060708090A0B0C85
:100200000D0E0F101112131415161718191A1B1CA6
:100210001D2F3130354C1E0F0500047F3F1F643207
:1002200014643214783C1E1E140A0505010902A14B
:100230000185020901A100050919012908150025F8
:1002400001950875018102050109300931158125E3
:100250007F95027508810609381581257F950175FE
:10026000088106050C0A38021581257F950175085D
:100270008106C0C005010980A101850319012AB7C3
:1002800000150126B700950175108100C0050C0905
:1002900001A101850419012AA002150126A00295D9
:1002A0000175108100C005010906A1018506050739
:1002B00019E029E715002501950875018102050758
:1002C000190029EF1500250195F075018102050837
:1002D0001901290595057501910295017503910193
:1002E000C00660FF0961A1010962150026FF0095A3
:1002F00020750881020963150026FF009520750806
:100300009102C005010906A101050719E029E715B9
:100310000025019508750181029501750881010587
:1003200007190029FF150026FF00950675088100B2
:10033000050819012905150025019505750191028A
:10034000950175039101C009025B00030100A0FA49
:10035000090400000103010100092111010001222B
:10036000440007058103080001090401000203009D
:10037000000009211101000122220007058203204B
:100380000001070503032000010904020001030026
:10039000000009211101000122B600070584032095
:1003A000000112010002000000082540554C011018
:1003B0000102000110034C00750064006400690034
:1003C0007400650000000C036400690030006900DF
:1003D000620000000403090435001E001F00200015
:1003E00021002200230024002500260027002D00E4
:1003F0002E002A002B0014001A0008001500170018
:100400001C0018000C00120013002F0030003100F7
:10041000394104001600070009000A000B000D0016
:100420000E000F00330034002800E1001D001B0007
:1004300006001900050011001000360037003800D2
:100440005232E000E300E2002C00E600504151424D
:100450004F3100000000000029003A003B003C0042
:100460003D003E003F004000410042004300440088
:1004700045004C0001000100520001000100010094
:10048000010001000100010046004A004D0001008A
:100490000100500051004F00010001000100010067
:1004A000010001004B004E0001000100AC00AE0055
:1004B000AB000100AA00A900A800010049004C00FF
:1004C00001000100010001000100010001007600AF
:1004D0000100000000000000010001000100010017
:1004E0000100010001000100010001000278047810
:1004F0000378010020782178237825782778010077
:100500000100010001000100010001000100007C68
:100510000100227824782678287801000100010063
:1005200001000100010001000100010001000100C3
:1005300001000100010001000100010001000100B3
:1005400001000100010001000100010001000100A3
:100550000100000000000000010001000100010096
:100560000100010001000100010001000100010083
:100570000100010001000100010001000100010073
:100580000100010001000100010001000100010063
:100590000100010001000100010001000100010053
:1005A0000100010001000100010001000100010043
:1005B0000100010001000100010001000100010033
:1005C0000100010001000100010001000100010023
:1005D0000100000000000000FFAA7F5540222325F3
:1005E0002628292A2C2D2F3032333536383A3B3DF8
:1005F0003E4042434547494A4C4E50515355575946
:100600005A5C5E6062646668696B6D6F7173757762
:10061000797B7D7F81838587898A8C8E9092949661
:10062000989A9C9E9FA1A3A5A7A8AAACAEAFB1B370
:10063000B4B6B8B9BBBCBEBFC1C2C3C5C6C7C9CAC0
:10064000CBCCCDCED0D1D2D2D3D4D5D6D7D7D8D982
:10065000D9DADADBDBDBDCDCDCDCDCDDDDDDDDDCE0
:10066000DCDCDCDCDBDBDBDADAD9D9D8D7D7D6D5F2
:10067000D4D3D2D2D1D0CECDCCCBCAC9C7C6C5C3B4
:10068000C2C1BFBEBCBBB9B8B6B4B3B1AFAEACAA01
:10069000A8A7A5A3A19F9E9C9A98969492908E8CB1
:1006A0008A89878583817F7D7B79777573716F6D8B
:1006B0006B6968666462605E5C5A59575553515065
:1006C0004E4C4A4947454342403E3D3B3A38363519
:1006D0003332302F2D2C2A292826252322000101F0
:1006E00001010101010101020202020202020202F1
:1006F00003030303030303030404040404040405C1
:100700000505050506060606060707070707080884
:100710000808090909090A0A0A0B0B0B0C0C0C0D35
:100720000D0D0E0E0E0F0F0F1010111111121213CE
:10073000131414151516161717181819191A1A1B49
:100740001B1C1D1D1E1E1F202021222223242425A8
:100750002626272829292A2B2C2D2D2E2F303132E1
:1007600032333435363738393A3B3C3D3E3F4041F1
:1007700042434445464748494A4C4D4E4F505153D9
:1007800054555658595A5B5D5E5F61626465666890
:10079000696B6C6D6F7072737577787A7B7D7E8014
:1007A00082838587888A8C8E8F91939596989A9C60
:1007B0009EA0A2A3A5A7A9ABADAFB1B3B5B7BABC74
:1007C000BEC0C2C4C6C9CBCDCFD1D4D6D8DBDDDF45
:1007D000E2E4E7E9EBEEF0F3F5F8FAFDFF001124AF
:1007E0001FBECFEFDAE0DEBFCDBF11E0A0E0B1E089
:1007F000E6E0F7E502C005900D92A43AB107D9F7FB
:1008000022E0A4EAB1E001C01D92AC3FB207E1F7DB
:100810000E946A0A0C94812B0C940000A8E0B0E0BE
:10082000E4E1F4E00C94F92AFC018481882309F4C2
:100830004DC67F0121E040815181628173819581A4
:100840000E94B7288C01F7019581992309F4BAC158
:10085000980137572038310508F032C1003108F0CF
:10086000E2C28FEF93E00E94DE298111DCC238E200
:10087000A32E32E0B32E002379F0A114F4E0BF06DA
:1008800009F4D1C2C5010E94DE29811101C00150C5
:100890002FEFA21AB20AEFCFCE0101962C0188E009
:1008A000F20111928A95E9F72AE0322E85010F5F55
:1008B0001F4FC5010E94DE2989831A82882309F40B
:1008C000B2C2813009F041C06501F2E0CF0ED11C07
:1008D000C8010E94DE298A83882309F4A4C29FEFFD
:1008E000980F933060F423E0A20EB11CC6010E9461
:1008F000DE298B83882309F496C21C8229C08430A8
:1009000031F54E0133E0830E911C02E010E05601F8
:100910008FEFA81AB80AC6010E94DE29F40181935C
:100920004F01882309F47FC28C3741F4E2E0F0E004
:10093000EC0FFD1FE00FF11F10820AC00F5F1F4F69
:1009400065010730110519F76EC2580101C0560143
:100950008201F8012081222309F4A8CF213009F077
:1009600053C08181813081F46801F2E0CF0ED11C47
:10097000F8018281893319F460E570E002C060E01B
:1009800070E00E94DE2615C0823049F46801F2E072
:10099000CF0ED11CF80182810E9427260AC0833025
:1009A00051F46801F2E0CF0ED11CF80182810E945F
:1009B000CD25860182C0843019F00F5F1F4F7DC0A6
:1009C000F80122810E5F1F4F80E090E030E020535D
:1009D00031092A30310568F4389EA001399E500D46
:1009E0001124C901840F951F0F5F1F4FF80120814B
:1009F000EDCF009709F461C0EFE9FFE03197F1F71F
:100A000000C000000197F5CFE22FF0E0EA56FE4F5C
:100A10002490822F86958695869590E0FC01EA5772
:100A2000FE4F64902770712C022E02C0759467945B
:100A30000A94E2F7F1E06F227724FC01EA58FE4FB6
:100A40008490912C022E02C0959487940A94E2F728
:100A500031E083229924FC01EA59FE4FC490D12C45
:100A600002C0D594C7942A95E2F781E0C822DD241C
:100A70006114710419F081EE0E94272681149104FB
:100A800019F086EE0E94272660E070E0822D0E9419
:100A9000DE268114910419F086EE0E94CD256114A2
:100AA000710419F081EE0E94CD25C114D10429F002
:100AB00060E070E08CE20E94DE260F5F1F4F49CF9E
:100AC0000230E8E71E0709F470C058F4011528E762
:100AD000120791F0013038E7130709F073C080E086
:100AE0000CC0043088E7180709F446C068F00530E8
:100AF000F8E71F07C9F066C084E00E948D2080914E
:100B0000DD020E9462208FC18091DD02982F9695B0
:100B10009695969549F1915E990F990F990F877067
:100B2000892B8093DD0214C09091DD02892F869578
:100B3000869586958F5F8F719770853008F03FC0DE
:100B4000880F880F880F892B8093DD028091DD024A
:100B5000887F91E009F490E08091DD0290FB80F9BC
:100B60008093DD020E9462208091DD028695869549
:100B700086950E94C51F57C12091DD02822F869560
:100B800086958695482F50E04430510554F48F5F88
:100B9000982F990F990F990F822F8770892B809327
:100BA000DD028091DD028160DBCF8091DD0280FF7C
:100BB00003C00E94A72037C10E94B42034C1909383
:100BC000DD02C4CFF801E851FC47E730F10508F435
:100BD000E6C0992309F453C410929B029801305740
:100BE0002332310508F00CC184E090E00E94EC292A
:100BF0009093A3028093A202F801E150F047E23201
:100C0000F10520F4EA5AFF4F0C94DD2A8091A202EC
:100C10008160ACC08091A3028860B4C08091A202C0
:100C20008260A4C08091A20220C08091A20288604C
:100C30009DC08091A3021EC08091A3028260A2C0C9
:100C40008091A202806192C08091A20280628EC0D7
:100C50008091A20280648AC00E94B3248091A20283
:100C6000806884C08091A202886084607FC0809187
:100C7000A3028260816086C08091A2028E7F76C0CE
:100C80008091A302877F7EC08091A2028D7F6EC07B
:100C90008091A20220C08091A202877F67C08091CC
:100CA000A3021EC08091A3028D7F6CC08091A2021E
:100CB0008F7E5CC08091A2028F7D58C08091A2027D
:100CC0008F7B54C00E94B3248091A2028F774EC0C4
:100CD0008091A202877F8B7F49C08091A3028D7F84
:100CE0008E7F50C08091A20282FB222720F991E0E2
:100CF000922790FB82F990FB83F938C08091A30280
:100D0000982F909591708E7F892B90FB81F93AC036
:100D10008091A20286FB222720F991E0922790FB86
:100D200086F924C00E94B3248091A20287FB222767
:100D300020F991E0922790FB87F918C061E001C08B
:100D400060E08EE090E00E94022A1EC08091A20224
:100D500084FB222720F991E0922790FB84F906C0BA
:100D60008091A202982F909590FB80F98093A20227
:100D70000BC08091A30283FB222720F991E09227E8
:100D800090FB83F98093A3026091A2027091A30269
:100D900084E090E00E94202A0E94B32444C0E858D6
:100DA000FF4F0C94DD2A06E221EE41EE6AE17CE77A
:100DB00005C007E225EE45EE6BE17CE7C7010E9426
:100DC0001D1E31C006E221EE40EE68E17CE7F6CF61
:100DD00007E225EE44EE69E17CE7F0CF06E221EE82
:100DE00042EE6CE17CE7EACF07E225EE46EE6DE1EC
:100DF0007CE7E4CF08E221E045EE6EE17CE7DECF60
:100E0000809146020631FCE71F07F9F48A7A91E0E7
:100E100009F490E09093A60181112FC389E20E940A
:100E2000521D0E94821980911B02877009F44EC3E3
:100E3000F7018581882309F449C38091A30282FFC9
:100E400045C382E00E94D41941C38272F801E05286
:100E5000F847EB30F10508F05CC0E158FF4F0C9407
:100E6000DD2A8091D50280FF19C0282F2E7F209384
:100E7000D5023091D6024091D7025091D8026091AC
:100E8000D9027091DA028091DB029091DC020E941B
:100E900052271092AA020E94F320C5CF816080934E
:100EA000D50261E0869586950E94AC27BCCF882349
:100EB00029F00E94F827B7CF8823D9F30E9403288E
:100EC000B2CF882329F00E942A27ADCF8823D9F3F7
:100ED0000E943427A8CF882329F00E941027A3CF8F
:100EE0008823D9F30E941D279ECF882329F00E94D2
:100EF000F62699CF8823D9F30E94032794CF88231D
:100F000029F00E9478278FCF8823D9F30E94922757
:100F10008ACF0737FCE71F0711F481E0CCC20837FE
:100F20002CE7120709F4C6C29801205E3245203230
:100F30003105A8F4911115C00F7181E090E09C017A
:100F400002C0220F331F0A95E2F78901622F83E066
:100F500090E00E94022A802F0E948D2464CF992362
:100F6000E9F103303CE7130729F148F401159CE748
:100F7000190791F00130ECE71E0711F12FC00B3576
:100F8000FCE71F0741F10C352CE71207E1F00A35A9
:100F90001C4721F581E020C00E94B3248FEF94E329
:100FA000ECE081509040E040E1F700C000000E947A
:100FB0009D1C39CF6FEF7FEF80E090E00E94202AE8
:100FC0000E946C2930CF8091A30282FB882780F990
:100FD00091E0892701C080E00E94EB19F70185812B
:100FE00000811181882349F0C8010E94CC23D82EAA
:100FF000682FC8010E943C2404C0C8010E94082434
:10100000D82EB8018D2D0E942C180E943A18D82E87
:10101000192FA82EF7010581C680C2949FE0C9222E
:1010200080911B02877001F10023F1F0812F807FF6
:10103000803469F080E28D0D8830B0F0812F807EA1
:10104000803229F4F1E0FD1578F4CC2069F080912C
:10105000A30282FF09C082E00E94D41980911B0282
:101060008770BB24B3948111B12C912E92948FE0A0
:101070009822892D90E08C30910508F0D6C1FC01B2
:10108000E657FF4F0C94DD2A812F807F1F70882345
:1010900011F01295107F0023B9F0112309F4B3C1A8
:1010A00080E28D0D883010F0A11006C090914602AC
:1010B000192B1093460205C090911D02192B109315
:1010C0001D020E9482199FC18D2D0E94CD251123E2
:1010D00009F4ABC180E28D0D883088F1AA2079F146
:1010E000109590911D02192310931D022BC0812F82
:1010F000807F1F70803211F01295107F8D2DAA20F5
:1011000029F021E0A21609F44CC057C08091A30237
:1011100082FD1BC0002369F0112339F09091460233
:10112000192B109346020E94821980E00E94272604
:101130007CC180E00E94CD25112309F476C1812F66
:101140000E947B190E94821970C1002381F0CC207B
:10115000C1F131E0C31269C190911C02812F892332
:10116000181709F462C1192B10931C025EC1C1103B
:101170005CC1812F0E94E42480911C02912F98234E
:1011800029F0912F9095892380931C022091A7012B
:10119000812F822309F449C1109521232093A701AF
:1011A00044C1002329F085E08C1508F43EC109C034
:1011B00094E09C1508F439C115C0002331F0C1102A
:1011C00022C1812F0E94EB2430C1CC2059F08933F9
:1011D00009F028C1EFEFF7EE23E0E150F0402040A6
:1011E000E1F71EC1812F0E94E4241FC1812F869543
:1011F0008695837019F0813061F017C1002321F0CA
:101200008D2D912F937002C080E090E00E94AE1D62
:1012100012C1002321F08D2D912F937002C080E028
:1012200090E00E94891D07C1602F8D2D0E94F5243A
:1012300002C1812F8370A9F50111FBC04D2D42958C
:1012400046954770440F440F8D2D8F7090E09C01A0
:10125000042E01C0220F0A94EAF7D4FE08C08FE0E2
:1012600090E001C0880F4A95EAF7809501C080E0C0
:10127000169516951370123069F088F49091B001AC
:10128000113019F0822B892302C0922B892B0E94E6
:101290008D24CFC0822B9091B0018927F8CF822B6B
:1012A000F6CF002319F0812F817001C08695882325
:1012B00009F4BFC04D2D429546954770440F440F29
:1012C0008D2D8F7090E09C01042E01C0220F0A9496
:1012D000EAF7D4FE08C08FE090E001C0880F4A957D
:1012E000EAF7809501C080E01695169513701230CC
:1012F00059F078F49091B101113019F0822B8923C3
:1013000009C0922B892B06C0822B9091B1018927AD
:1013100001C0822B0E9471248CC01F70002339F001
:10132000812F0E9481248D2D0E94EB2482C08D2D5F
:101330000E94E424812F0E9474247BC08D2D32EF03
:10134000A31681F13A1538F090EFA91659F0E1EFA4
:10135000AE1619F154C0F3EFAF1659F124EFA216EF
:10136000C1F04DC0002381F034E03C1508F45DC0AD
:101370001F7181E090E0012E01C0880F0A94EAF706
:101380009091B101892720C085E08C1508F44DC0EB
:10139000EFCF8091A30282FD1AC0002329F0812F94
:1013A0008F7120C00023D9F3812F8F710E94742484
:1013B0003CC0002341F01F7181E0012E01C0880F65
:1013C0000A94EAF701C080E00E9471242EC0002335
:1013D00061F0812F8F7198E0899F90011124236023
:1013E00020931B020E94812420C081E00E94D41916
:1013F000E1E0EC15D0F482E00E94D41916C000237D
:1014000021F0CC2061F28D2D91CECC2069F2893370
:1014100049F4FFEF27EE33E0F15020403040E1F790
:1014200000C000008D2D0E94CD2588EF890D8430ED
:1014300010F40E94D31DBB20A9F080911B0280FDF7
:1014400011C0F70115828695869586950E948124A4
:10145000C7010E940E0480911B0286958695869591
:101460000E94742420E0F7014081518162817381E0
:10147000848195810E94B72829C085E3D0CC0631AC
:101480008CE7180751F48091A601811104C089E20C
:101490000E94241DC6CC85E3FBCF07372CE712073B
:1014A00011F481E00BC008373CE7130709F03CCD8D
:1014B00082E004C082E00E94812402C00E94742461
:1014C00043E062E081E00E94EC1BADCC2896E2E1B3
:1014D0000C94152BA6E2B0E0E0E7FAE00C94F92AB0
:1014E00085B7806885BF85B7806885BF84B7877FEB
:1014F00084BF0FB6F894A8958091600088618093AE
:101500006000109260000FBE90E080E80FB6F89483
:1015100080936100909361000FBE81E08093110180
:1015200088E396E19093A5018093A4010E94A514FD
:101530000E94C4148091E20084608093E200789459
:101540008091D0018823A1F01091E9001F70909143
:10155000EC00892F817090FD80E8182B1092E90033
:101560008091E80083FD0E9489111F701093E900AB
:1015700082E084BD93E095BD9AEF97BD80936E00A5
:101580000E94041E811102C00E94871F00E211E028
:10159000A8E2EA2EA1E0FA2ED8018D918D018F3FAD
:1015A00011F00E946B17E016F106B1F708E211E0A6
:1015B000F0E3EF2EF1E0FF2EF80181918F018F3FD4
:1015C00011F00E946B17E016F106B1F788E0EDEB21
:1015D000F1E0DF01282F1D922A95E9F7E8EAF1E012
:1015E000DF011D928A95E9F780E090E00E94EC29E6
:1015F000853E9E4F21F40E94041E811163C065EE5A
:101600007EEF80E090E00E94202A60E082E090E09F
:101610000E94022A81E08093B00161E083E090E0C3
:101620000E94022A60E074E184E090E00E94202A97
:1016300060E086E090E00E94022A60E087E090E0AF
:101640000E94022A40E050E0BA0188E090E00E9447
:10165000142A60E083E290E00E94022A60E08CE0BD
:1016600090E00E94022A60E08DE090E00E94022A51
:1016700019821A821B821C821D821E821F8218867A
:1016800048E050E067E170E0CE0101960E94F22947
:1016900040E050E0BA018FE190E00E94142A80E01F
:1016A0000E94E51D0E94871F40E050E0BA018FE0D4
:1016B00090E00E94142A40E050E0BA0183E190E0FB
:1016C0000E94142A82E090E00E94DE298093B301F8
:1016D00084E090E00E94EC299093A3028093A20200
:1016E0000E948217EFEFF6E721E0E150F040204042
:1016F000E1F700C000000E9482178091BD0180FFC9
:1017000008C06FEF7FEF80E090E00E94202A0E94E7
:101710009D1C83E090E00E94DE290E948D24259A82
:101720002D9882E88093800089E1809381008FEF7B
:101730009FEF90938700809386000E94CC200E94A8
:10174000CC208091B20181117FC088E090E00E949E
:10175000E6294B015C0183E290E00E94DE29282FFC
:1017600030E040E050E060E070E080E090E000E2D7
:101770000E94302B282939294A295B292093D50238
:101780003093D6024093D7025093D8026093D90287
:101790007093DA028093DB029093DC022C7F09F0D5
:1017A00041C025E02093D5021092D6023FEF30933E
:1017B000D7023093D8021092D90230E04FEF5FEF9A
:1017C00060E00E94522788E090E00E94E6296B01C9
:1017D0007C0183E290E00E94DE29282F30E040E087
:1017E00050E060E070E080E090E00E94302BB22F8B
:1017F000A32FF42FE52F5B0197018601BC29A12BB4
:10180000F22BE32BB093D502A093D602F093D7022C
:10181000E093D8026093D902B092DA028093DB029F
:101820009093DC020E943E271092AA020E941D1C87
:101830008091D50280FF05C060E0869586950E9464
:10184000AC2781E08093B20184E091E090939F0205
:1018500080939E0278E1C72ED12CE0E15E2EBB245E
:10186000B394AA24A3948E010F5F1F4F8091D001DF
:10187000853009F040C08091D001853009F035C035
:101880008091D001843029F180E00E948D20109257
:10189000A40280E40FB6F894A895C09260000FBE31
:1018A0008093600083B7817F846083BF83B781604A
:1018B00083BF7894889583B78E7F83BF0FB6F894E3
:1018C000A89580916000886180936000109260000C
:1018D0000FBE0E948217EDEBF1E08191811129C4C6
:1018E00091E0E53CF907C9F7C6CF0E94B3240E94F6
:1018F000CC200E94D31D0E94821754EBE52E51E0AC
:10190000F52E6DEB862E61E0962ED401F7019191B4
:101910008D91892721E0EC3BF20719F08823B9F378
:1019200005C0811103C00E94571932C0712CD40127
:101930002D904D01F7013080322409F1612C4424AF
:101940004394832D8421A1F069A27AA20E94EF1C06
:101950009CA38BA3ADA291E0822D842109F490E099
:101960009EA349A15AA16BA17CA18DA10E94DC2854
:101970006394440CF8E06F12E4CFD7012C92739477
:10198000BFEFEB1AFB0AE8E07E12D1CF0E94E31C06
:101990008091AA02882309F4ABC08091A902E0914A
:1019A000D502E695E695E81BE093F802823059F4FB
:1019B000F0E0E95DFD4FE491EE2EF12C49E7842E35
:1019C00040E2942E70C0863059F4F0E0EC5DFD4F9B
:1019D000E491EE2EF12C39E6832E30E2932E63C093
:1019E000893061F4E695F0E0EF5DFD4FE491EE2E75
:1019F000F12C2BEE822E22E2922E55C08F3061F414
:101A0000E695F0E0E25EFD4FE491EE2EF12C90E9D8
:101A1000892E92E2992E47C0853159F4F0E0E55EB7
:101A2000FD4FE491EE2EF12C84E4882E82E2982E74
:101A30003AC08831F9F0833249F4E9E1F2E0E59007
:101A4000F490B2E38B2EB3E29B2E2DC08432D1F002
:101A5000853209F58E2F63E00E94A92AE92FF0E074
:101A6000EA5EFD4FE491EE2EF12CABE08A2EA1E26E
:101A70009A2E19C0E8E2EE2EF12CFCEC8F2EF1E24A
:101A80009F2E11C064EFE62EFF24F3947DE9872E8C
:101A900071E2972E08C040EDE42E47E0F42E58E6A0
:101AA000852E50E2952E8091F902882361F01092E4
:101AB000F9020E94EF1C9093F7028093F6021092B5
:101AC000FB021092FA020E94EF1CE091F602F091E4
:101AD000F7028E1B9F0B8F3F9F4750F4EE0EFF1EA9
:101AE000F092F702E092F60286EF92E0F401099597
:101AF00086E0E3E9F2E0D80101900D928A95E1F7E2
:101B000070909402F09095029090960280909702C7
:101B1000E09098021092950210929602109297020D
:101B200010929802F11003C0992009F44BC08091E3
:101B30009102909192020E94D41C9C0190918C027F
:101B4000992309F41CC325313105E0F19F3F19F0B9
:101B50009F5F90938C02FF2061F00E94ED1E1F1486
:101B600014F491E001C09FEF899F802D1124809390
:101B70009502992061F00E94ED1E191414F09FEF58
:101B800001C091E0899F802D11248093960280915D
:101B900095028823B9F060909602662099F00E9421
:101BA0000D1F882319F08093950202C0B092950210
:101BB000862D0E940D1F882319F08093960202C083
:101BC000B0929602811003C0EE2009F44BC08091C0
:101BD0008F02909190020E94D41C9C0190918D02E2
:101BE000992309F4D1C221353105E0F19F3F19F065
:101BF0009F5F90938D02882061F00E94CB1E181485
:101C000014F491E001C09FEF899F802D11248093EF
:101C10009702EE2061F00E94CB1E1E1414F09FEF7D
:101C200001C091E0899F802D1124809398028091BA
:101C300097028823B9F060909802662099F00E947C
:101C40000D1F882319F08093970202C0B09297026B
:101C5000862D0E940D1F882319F08093980202C0E0
:101C6000B09298028091940287111AC080919502D7
:101C7000882311F08F1114C080919602882311F0EF
:101C800089110EC080919802882311F08E1108C02E
:101C900090919702992331F081E0981104C002C01D
:101CA00081E001C080E080FD15C080919502811126
:101CB0000FC08091960281110BC080919702811113
:101CC00007C081E090919802911103C080E001C0AB
:101CD00081E080FD0E94A11E7A82FB829C828D821F
:101CE000EE8286E0F801A3E9B2E001900D928A95B8
:101CF000E1F70E94D31D9091BC01891721F08093D8
:101D0000BC010E94E31C8091D001843009F0AECD6B
:101D100083E08093E9008091E80082FFA7CD809165
:101D2000E80085FF21C00E94051681111BC030E22A
:101D3000E32EF12C480109C08091F100D4018D936C
:101D40004D01B1E0EB1AF10869F08091E80085FDE2
:101D5000F3CF8091E8008B778093E8000E9405160E
:101D6000882399F391E001C090E08091E8008B779F
:101D70008093E800992309F479CD2981822F90E09E
:101D8000FC013197E331F10508F0CAC1EA56FF4F73
:101D90000C94DD2A1A828CE030C18A81823009F4E9
:101DA000E5C150F4813009F0BBC10E94E31C9B8364
:101DB0008C837D836E83B6C1833041F0843009F01B
:101DC000AFC11B821C821D821E82ACC16B81DE01F1
:101DD000149680E090E0262F30E0A901480F591FAB
:101DE0004830510508F09EC1E62FE80FF0E0E354BB
:101DF000FE4F40814D9301968C31910571F792C150
:101E00008A81823019F0853051F08AC16B817C81E2
:101E10008D819E810E94E32A0E94E01D83C18091F2
:101E2000DD0280FF03C00E94A72002C00E94B420F0
:101E30008091D50280FF0AC08091D5028E7F809369
:101E4000D5021092AA020E94F3206CC18160809397
:101E5000D50260E08695869583C04C816B818A812E
:101E60000E94971F9D8389C12D813E8132272327A0
:101E700032274C816B818A810E942B1F53C10E94A3
:101E8000521F50C18A81813081F5283099F0293064
:101E900039F18B81813009F045C18C81E4E08E9F5E
:101EA000C00111246FEF70E00E94B52A862F0E94B6
:101EB0008D2038C18B81813029F0823009F032C108
:101EC0001C8230C18091DD02869586958695FFEF54
:101ED0008F9FC0011124969587959695879574C01C
:101EE0008091DD020E9462201DC1823009F018C17C
:101EF000283009F43FC0293009F468C08B81823052
:101F0000F9F098F4813009F00DC18C812FEF829F98
:101F1000C00111246FEF70E00E94B52A462F20E027
:101F20006091D7028091D60222C08330E1F08430E4
:101F300009F0F8C020E04091D8026D818C8117C073
:101F40008C81882309F478CF8091D50281608093B9
:101F5000D50260E0869586950E94AC2760E08C8172
:101F60000E94AC27DFC08C818093D902DBC00E9425
:101F70004F23D8C08B818230E1F078F4813009F0B2
:101F8000D1C08091D802AFEF8A9FC00111246FEFBA
:101F900070E00E94B52A6C83C5C0833099F084300C
:101FA00009F0C0C08091D6028C838091D7028D83C6
:101FB000B9C08091D50280FF03C08695869504C084
:101FC00080E002C08091D9028C83ACC02091D50200
:101FD0003091D6024091D7025091D8026091D90237
:101FE0007091DA028091DB029091DC020E9452270C
:101FF00099C05A8297C0BA8288ED8B8393C0EA80D9
:10200000FB80FE24EF24FE248C80912C3801C70134
:10201000885D9D4F9301201B310B2815390508F071
:1020200081C0B8EDEB16B1E0FB0628F40E94DE2972
:10203000F301848303C0D30114961C92BFEFEB1A03
:10204000FB0AEFEF6E1A7E0AE2CFEA80FB80FE24E5
:10205000EF24FE248C80912C3801C701885D9D4FB0
:102060009301201B310B2815390508F05BC0F8EDF2
:10207000EF16F1E0FF0628F4D30114966C910E944C
:10208000022ABFEFEB1AFB0AEFEF6E1A7E0AE5CFCA
:102090000E941B1F47C084E08A8344C0EA80FB8003
:1020A000FE24EF24FE248C80912C3801C7018896F1
:1020B0009301201B310B28153905A0F5E114F2E03E
:1020C000FF0630F40E94DE29D30114968C9302C0DF
:1020D000F3011482FFEFEF1AFF0A2FEF621A720A60
:1020E000E5CFEA80FB80FE24EF24FE248C80912C37
:1020F0003801C70188969301201B310B281539053B
:1021000088F4E114A2E0FA0620F4F30164810E944D
:10211000022AFFEFEF1AFF0A2FEF621A720AE9CFC5
:102120008FEF898340E250E0B80182E00E94441CB6
:102130009DCB8091CF01882309F49DCBA0E1A9BD5F
:10214000B2E1B9BD09B400FEFDCF8091D8008F7D0A
:102150008093D8008091E00082608093E0008091BD
:10216000E00081FDFCCF0E94B32485CB87E290E0A4
:102170000E94DE291B821C821D828E83D3CF2B30CE
:10218000310508F0E5CC1ECD2B30310508F030CDFF
:1021900069CD8091D20187FF11C08091E80082FD56
:1021A00005C08091D0018111F8CF11C08091E80065
:1021B0008B770BC08091D001882349F08091E80093
:1021C00080FFF8CF8091E8008E778093E800089533
:1021D000982F973068F59093E900981739F070912F
:1021E000EC002091ED005091F00003C0242F762FD9
:1021F00050E021FD02C09F5FECCF3091EB003E7FAD
:102200003093EB003091ED003D7F3093ED00309145
:10221000EB0031603093EB007093EC002093ED0005
:102220005093F0002091EE0027FDE5CF80E0089567
:102230008F708093E90081E008952091D80130915A
:10224000D9012617370748F06115710539F4209137
:10225000E8002E772093E80001C0B901FC0120E0DE
:102260006115710579F18091D0018823F1F18530F4
:10227000F1F18091E80083FD3CC08091E80082FD8F
:102280002EC08091E80080FFEBCF2091F300809179
:10229000F20090E0922B6115710551F088309105A4
:1022A00038F421912093F100615071090196F3CF28
:1022B00021E0089709F020E08091E8008E77809374
:1022C000E800CECF2111CFCF0AC08091D001882362
:1022D00061F0853061F08091E80083FD0AC0809153
:1022E000E80082FFF2CF80E0089582E0089583E065
:1022F000089581E0089543E050E0BC0184E00E942D
:10230000441C089546E050E0BC0184E00E94441C57
:102310000895AAE2B0E0EFE8F1E10C94082BE2EDB9
:10232000F1E08AED91E02091F10021938E179F0753
:10233000D1F78091D301833009F463C030F4813048
:1023400071F0823009F4A2C0B9C08A3009F48EC09D
:102350008B3009F46EC0893009F0B0C020C0809184
:10236000D201813A09F0AAC08091E800877F80936A
:10237000E8008091D6019091D701892B21F468E083
:1023800086EC91E003C060E080E090E070E00E94A5
:102390001D118091E8008B778093E8008FC08091B9
:1023A000D201813209F08AC08091D6019091D70183
:1023B000009719F0029709F081C08091E800877FAB
:1023C0008093E8008091E80082FD05C08091D001F3
:1023D0008111F8CF73C02091F3008091F20090E05A
:1023E000922B029731F48091F100813011F0863008
:1023F00021F48091F10080930F018091E8008B77A8
:1024000059C08091D201813A09F058C08091D6011B
:102410009091D701892B09F051C08091E800877F06
:102420008093E8008091E80080FFFCCF809110014C
:102430003CC08091D201813209F040C08091D60128
:102440009091D701892BD1F58091E800877F809307
:10245000E8000E94C91081E09091D401911101C05F
:1024600080E0809310010E94B32428C08091D201A3
:10247000813221F58091E800877F8093E8000E94F7
:10248000C9108091D50180930E0118C08091D201AE
:10249000813AA1F48091E800877F8093E8008091E1
:1024A000E80080FFFCCF80910E018093F1008091C5
:1024B000E8008E778093E8000E94C9108091E800C0
:1024C00083FFE7C18091D2019091D301492F50E061
:1024D0004A30510508F0DDC1FA01E755FF4F0C9471
:1024E000DD2A803821F0823809F0D3C108C08091FC
:1024F000CE019091CF01992389F082600FC0809125
:10250000D6018F70873008F0C4C18093E9008091B4
:10251000EB0085FB882780F91092E9009091E80094
:10252000977F9093E8008093F1001092F10071C1C1
:10253000282F2D7F09F0ADC1882319F0823061F07A
:10254000A8C18091D401813009F0A3C1933009F072
:1025500080E08093CF012EC08091D40181112AC0E8
:102560008091D6018F702FEF280F263008F091C18F
:102570008093E9002091EB0020FF1CC0933021F4F0
:102580008091EB00806214C09091EB009061909379
:10259000EB0021E030E0A90102C0440F551F8A95ED
:1025A000E2F74093EA001092EA008091EB00886025
:1025B0008093EB001092E9008091E800877F809380
:1025C000E8000E94C91065C1811163C11091D40156
:1025D0001F778091E3008078812B8093E3008091C6
:1025E000E800877F8093E8000E94C9108091E8008E
:1025F00080FFFCCF8091E30080688093E30011119D
:1026000002C082E001C083E08093D00142C18058C3
:10261000823008F03EC12091D4013091D5012C3D8B
:1026200053E0350779F583E08A838AE289834FB7DF
:10263000F894DE01139620E03EE051E2E32FF0E053
:1026400050935700E49120FF03C0E295EF703F5F85
:10265000EF708E2F90E0EA3010F0C79601C0C09660
:102660008D939D932F5F243149F74FBF8091E800F0
:10267000877F8093E8006AE270E0CE0101960E94B5
:102680001D11B5C08091D6019091D701432F5527D8
:1026900043305105A9F068F44130510509F408C1EF
:1026A0004230510509F0F5C08BE590E0E7E4F3E036
:1026B0004BC04132510529F14232510589F1E9C03F
:1026C000C901992781309105A1F058F0029709F0CE
:1026D000E0C0E4EBF3E0E4918E2F90E0E4EBF3E074
:1026E00030C0E4EDF3E0E4918E2F90E0E4EDF3E010
:1026F00028C0E6ECF3E0E4918E2F90E0E6ECF3E006
:1027000020C08330910508F0C4C0880F991FFC01D8
:10271000E75CFE4F0190F081E02D89E090E014C06D
:102720008330910508F0B5C0FC01EE0FFF1FED5C92
:10273000FE4F0190F081E02DDC01A05DBE4F8C9139
:1027400090E0009709F4A5C02091E800277F20932E
:10275000E8002091D8013091D9018217930708F43D
:102760009C0140E02115310589F18091D001882339
:1027700009F43DC08530D9F18091E80083FD37C070
:102780008091E80082FD2FC08091E80080FFEACFB1
:102790004091F3008091F20090E0942B21153105D7
:1027A00059F08830910540F444914093F1003196FE
:1027B000215031090196F2CF41E0089709F040E03D
:1027C0008091E8008E778093E800CCCF4111CDCF87
:1027D0000AC08091D001882351F0853041F080916A
:1027E000E80083FD04C08091E80082FFF2CF809171
:1027F000E8008B778093E8004CC0803809F049C02E
:102800008091E800877F8093E8008091D1018093D8
:10281000F1008091E8008E77D2CE81113AC080918C
:10282000D4019091D501992702979CF58091E800F9
:10283000877F8093E8001091D4011093D1010E940A
:10284000C910111106C08091E30087FD02C081E02C
:1028500001C084E08093D00142E061EC81E00E94FD
:10286000E81042E261EC84E00E94E81042E261EC90
:1028700082E00E94E81042E260EC83E00E94E810EF
:102880008091D001843011F081E001C082E080931A
:1028900011018091E80083FF10C08091E800877FDC
:1028A0008093E8008091EB0080628093EB0005C08C
:1028B00082E190E0E2EAF3E047CFAA96E3E00C94ED
:1028C000242B1F920F920FB60F9211242F933F9338
:1028D0004F935F936F937F938F939F93AF93BF9328
:1028E000CF93DF93EF93FF93C091E900CF70809176
:1028F000EC00D82FD17080FDD0E81092E9008091D3
:10290000F000877F8093F00078940E9489111092E4
:10291000E9008091F00088608093F000CD2BCF70AB
:10292000C093E900FF91EF91DF91CF91BF91AF91FB
:102930009F918F917F916F915F914F913F912F91D7
:102940000F900FBE0F901F901895E8EDF0E080817A
:102950008E7F80831092E2001092DA001092E100E4
:10296000A0EEB0E08C9181608C9380818F77808322
:1029700019BCA7EDB0E08C918E7F8C9380818F7E07
:1029800080831092C5010895A0E0B0E0EAECF4E184
:102990000C94032BC8EDD0E088818F7E8883E7ED0F
:1029A000F0E080818160808384E082BF81E0809359
:1029B000C50188818E7F888302EE10E0F8011082C5
:1029C0001092DA0081EEC82ED12CF6011082888197
:1029D0008F77888388818068888388818F7D8883CA
:1029E00019BC1092D0011092D1011092CF01109217
:1029F000CE0190EEE92EF12CF70180818B7F808350
:102A000088818160888342E060E080E00E94E81075
:102A1000F60180818E7F8083F801808181608083D0
:102A2000808188608083F70180818E7F80838881A8
:102A300080618883CDB7DEB7E8E00C941F2B1F922E
:102A40000F920FB60F9211242F933F934F935F93E2
:102A50006F937F938F939F93AF93BF93EF93FF9366
:102A60008091E10082FF09C08091E20082FF05C0F1
:102A70008091E1008B7F8093E1008091DA0080FFFC
:102A80002AC08091D80080FF26C08091DA008E7F16
:102A90008093DA008091D90080FF18C080E189BD61
:102AA00082E189BD09B400FEFDCF81E08093D001B1
:102AB0008091C50181110FC00E94A5140E94C41409
:102AC0008091E20084608093E20005C019BC1092FE
:102AD000D0011092C5018091E10080FF1AC0809161
:102AE000E20080FF16C08091E2008E7F8093E200BA
:102AF0008091E20080618093E2008091D800806242
:102B00008093D80019BC85E08093D00183E0809346
:102B100011018091E10084FF37C08091E20084FFC1
:102B200033C080E189BD82E189BD09B400FEFDCFDB
:102B30008091D8008F7D8093D8008091E1008F7EB6
:102B40008093E1008091E2008F7E8093E20080918B
:102B5000E20081608093E2008091D101882311F02E
:102B600084E007C08091E30087FD02C081E001C0DE
:102B700083E08093D0018091D001843011F081E016
:102B800001C082E0809311018091E10083FF2CC09D
:102B90008091E20083FF28C08091E100877F8093CD
:102BA000E10082E08093D0011092D1018091E10098
:102BB0008E7F8093E1008091E2008E7F8093E2001F
:102BC0008091E20080618093E20042E060E080E07A
:102BD0000E94E8108091F00088608093F00081E00E
:102BE0008093110180931001FF91EF91BF91AF91FC
:102BF0009F918F917F916F915F914F913F912F9115
:102C00000F900FBE0F901F9018952091E400309107
:102C1000E50095E64091EC00842F817040FF23C0D1
:102C20008091E80080FD1DC08091D001882399F03B
:102C3000853099F08091EB0085FD11C04091E40052
:102C40005091E5002417350729F3915011F09A01AE
:102C5000E1CF84E0089582E0089583E0089581E063
:102C6000089580E008954091E80042FFDDCF089587
:102C700080E008959091A20292FF10C041E0282FB9
:102C80002471243009F040E031E0282F28712830E9
:102C900009F030E0431711F02CE0822793FF10C0B9
:102CA00041E0282F2471243109F040E031E0282F41
:102CB0002871283109F030E0431711F02CE0822709
:102CC0003091A30230FF10C051E0282F2171213034
:102CD00009F050E041E0282F2871283009F040E049
:102CE000541711F029E0822731FF10C041E0282F4E
:102CF0002171213109F040E031E0282F287128317D
:102D000009F030E0431711F029E0822794FD877E17
:102D100008958238910569F1B0F48133910509F481
:102D200075C048F48932910509F467C08A3291056B
:102D300009F471C008958533910509F459C08933A8
:102D40009105B9F00895833E910589F138F4803EEC
:102D50009105D1F0823E910529F10895863E9105B5
:102D6000C9F1873E9105D9F1843E910509F06CC007
:102D700027C02091A20220FD57C021FD55C02091FF
:102D8000A30223FD5BC008958091A20280FD48C08C
:102D90008091A30280FF48C08091A20284FD46C0BA
:102DA00083EE51C08091A20282FF3CC0F5CF80919A
:102DB000A20282FD37C08091A30280FD35C0ECCF16
:102DC0008091A30281FF36C08091A20284FD2EC0B3
:102DD00087EE39C08091A20283FF2AC0F5CF80918F
:102DE000A20283FD25C08091A30281FD23C0ECCF08
:102DF0008091A20285FD22C01FC08091A20285FDA4
:102E00001BC08091A30283FF19C00AC08091A20257
:102E100086FD16C017C08091A20286FD13C010C0A7
:102E200089E311C082EE0FC080EE0DC080E00BC0C0
:102E300086EE09C084EE07C085E305C089E203C0C1
:102E40008AE201C081E390E008959091460280916A
:102E50001D02892B90911C029923E1F0892B9091FE
:102E60001001913041F49091A20297FF04C09EE1BD
:102E700026E532E003C096E02EE432E0F90120E0DE
:102E8000915028F031913323D9F32F5FF9CF2111DD
:102E900010921C02089520911A029091E10157E0CE
:102EA0002917A9F030E0529FF001539FF00D112433
:102EB000EE51FE4F7181761306C07081781303C006
:102EC0007581741306C02F5F3F4F2770E9CF80E0F4
:102ED000089581E00895F894E82FE295EF70F0E00E
:102EE00031A1282F2F7081E090E001C0880F2A9532
:102EF000EAF7982F9095932391A392A1892B82A30F
:102F000078940895A8E0B0E0E8E8F7E10C94002B8D
:102F1000AE014F5F5F4F7A0188E0FA0111928A9506
:102F2000E9F700E211E06A01AA24A394B12CF801A8
:102F300080818F3F09F441C0F894E82FE295EF704B
:102F4000F0E021A18F70A50102C0440F551F8A95A2
:102F5000E2F7CA01922F982B91A392A18095892321
:102F600082A3789400C0E8E2F1E0912C31E0219155
:102F70002F3F89F0A22FA295AF70B0E090968C9170
:102F800090E02F7002C0959587952A95E2F780FD15
:102F900002C0832F01C080E0982A330F51E0E03354
:102FA000F50729F7F80180818F3F11F00E946B1718
:102FB000F0EAFA95F1F7F60190820F5F1F4FFFEFED
:102FC000CF1ADF0A41E00832140709F0B0CF48E019
:102FD00050E0B70188EA91E00E94742B892B91F0B0
:102FE00088E0F701A8EAB1E001900D928A95E1F737
:102FF00081E080934B020E94EF1C90934A028093E1
:1030000049020CC080914B02882341F08091490213
:1030100090914A020E94D41C059710F480E018C0D9
:1030200048E050E068EA71E08DEB91E00E94742B7B
:10303000892B59F088E0E8EAF1E0ADEBB1E00190CE
:103040000D928A95E1F781E001C080E010924B0279
:103050002896EBE00C941C2B783048F4683038F458
:10306000843028F4462F672F0E94971F089580E030
:1030700090E008951F93CF93DF930E948916EC018F
:10308000C11580E5D807E8F5C11590E4D90708F027
:10309000A8C0C03ED10530F5CD3CD10508F094C0A4
:1030A000C83AD10578F4C53AD10508F083C0C130DB
:1030B000D10509F47CC008F4F2C0C430D10508F091
:1030C000F1C0EDC0C33CD10508F0E9C0C85AD0E05A
:1030D000CC0FDD1FCE5BDE4F0990D881C02DCE0115
:1030E0009464E1C0C11580E2D80708F0CBC0C115D7
:1030F00091E0D90708F06BC0C83ED10508F4D2C0F2
:10310000CEC0C03682E5D80728F5C03492E5D9078D
:1031100008F079C0C03282E5D80708F06CC0C1154C
:1031200092E5D90708F481C04C2F4695469580E278
:10313000489FA0011124C37021E030E0C90102C002
:10314000880F991FCA95E2F7EA01C82BD92BCE0147
:103150009D68A9C0C03A82E5D807B8F48C2F8F715A
:10316000C03892E5D90708F07BC08695869590E235
:10317000899F90011124C37081E090E002C0880F04
:10318000991FCA95E2F79A6868C0C03C82E5D807E3
:1031900008F46DC0C03E92E5D90708F080C0CF7139
:1031A000DD27DC2FCC27CE01806F906A7CC081E0C8
:1031B00090E079C0C55AD0E0C15CDE4F8881C82F4D
:1031C000D0E0CE0190646FC0CE0190656CC08D2FB1
:1031D0000E943A16182FCE0199270E9489161F7156
:1031E0005CC0CE0199270E948916CC27DF70D06A77
:1031F0008C2B9D2B58C0CF71D0E0DC2FCC27CE017B
:10320000816F906A50C08C2F8F718695869590E261
:10321000899F90011124C37081E090E002C0880F63
:10322000991FCA95E2F79C6818C08C2F8F710E9475
:103230003A1695E0D695C7959A95E1F7CF70D0E00C
:10324000DC2FCC27282F30E084FF05C084E0220F3C
:10325000331F8A95E1F7D069CE01822B932B23C0CF
:1032600090E0D82FCC27CE01846F906A1CC08C2FA1
:103270008F710E943A168F7190E0D82FCC27CE0123
:10328000906211C08D2F8F710E943A16182FCE01B7
:1032900099270E9489161F719062912B04C080E0CB
:1032A00090E001C0CE01DF91CF911F910895A6E07B
:1032B000B0E0EDE5F9E10C94072B0E94EF1C8C01C6
:1032C00080914702909148020817190781F01982EE
:1032D0001A820E94EF1C682F49815A81792F80E061
:1032E00090E00E94DC281093480200934702269643
:1032F000E4E00C94232B80959091460289238093DF
:103300004602089580911001813051F58091A2020A
:1033100087FF26C00E9425178093550240E250E0A7
:103320006EE172E084E592E00E94742B892BD9F162
:1033300080E2E4E5F2E0AEE1B2E001900D928A9520
:10334000E1F7E0919E02F0919F02309761F186E0F3
:10335000809354020480F581E02D84E592E022C040
:103360000E94251780934C0248E050E06EE372E023
:103370008CE492E00E94742B892BA9F088E0ECE4A5
:10338000F2E0AEE3B2E001900D928A95E1F7E091B0
:103390009E02F0919F02309731F00280F381E02D80
:1033A0008CE492E00995089590911B028095892301
:1033B00080931B02282F277069F4981759F0909179
:1033C000A30292FF07C08695869586950E94742475
:1033D00010921B0208959091A30292FB222720F9DC
:1033E000281779F080FB92F99093A3026091A202D2
:1033F0007091A30284E090E00E94202A82E00E9463
:10340000D419089580911A029091E101891719F059
:103410008F5F8770FBCF0895CF93DF938091E0019A
:1034200082958F7009F04EC08091DF01882309F4E6
:1034300049C080911A024091E1015091DB016091F5
:10344000DA01C091DC01D091DD0177E08417D1F180
:1034500090E0789FF001799FF00D1124DF01AE51CB
:10346000BE4F14962C911497222349F111962C915A
:103470001197251324C02C91261321C015962C9149
:10348000159721111CC012962D913C9113972C1B5E
:103490003D0B283C310598F48091E0018F708061EC
:1034A0008093E001E851FE4F80818F7080618083BE
:1034B0008AED91E00E940E040E94021A03C0019658
:1034C0008770C4CFDF91CF910895A4E1B0E0EBE61F
:1034D000FAE10C94FF2A8C0186E0F801DE011F96C8
:1034E00001900D928A95E1F7F8018481E5809AEDCB
:1034F000892E91E0992E9091DE01911120C08823B0
:1035000009F463C1EE2009F442C0C8010E9490246E
:10351000F82E8823E1F187E0F801D40101900D92A3
:103520008A95E1F78091DE01813031F48091DA01F2
:103530009091DB010E94FB230E940C1A48C1F80104
:10354000D080C180A280B380F090DF012091DC01A7
:103550003091DD01FF2009F4E7C0A501421B530BA8
:10356000483C510508F09DC0882309F430C1809182
:10357000E001282F207F9091DB01222361F09C1530
:1035800009F460C0C8010E949024811163C0C80181
:103590000E940E041AC19C1113C09091DA019D1172
:1035A0000FC0E1100DC08F7080618093E0018AED43
:1035B00091E00E940E048091E001F801868303C12E
:1035C000E1103AC040E06C2D8D2D0E944B1740E079
:1035D0006C2D8D2D0E944B17E82E8111F4C0DF86D3
:1035E000C88A8F8598890E94FB23292F22952F70E6
:1035F000243020F49F70223028F009C02A50223055
:1036000080F014C0992349F0811107C013C0992399
:1036100021F0F8019681907F69F0805E883030F467
:1036200009C0803F38F0815F833020F0C8010E94DC
:103630000E04EF2CFE2CCBC08091E00181608093C2
:10364000E001C1C09091DA019D119CCFE1109ACFA9
:10365000F80198C0EE2009F49ACF2091E001822F62
:1036600082958F7090E002978CF08091DA019091B2
:10367000DB0199878887BB86AA868091DE018C87CB
:103680001D862E87CE0108960E940E0487E0F80161
:10369000AAEDB1E001900D928A95E1F70E940C1A13
:1036A00094C09091E001292F207F51F48AED91E0A0
:1036B0000E940E0487E0F40111928A95E9F783C015
:1036C000882309F484C08091DB018C110CC08091A7
:1036D000DA018D1108C0E11006C0F8019683C80117
:1036E0000E940E046AC0C8010E949024882309F435
:1036F0004ECFEE2009F44BCF2091E001822F82952E
:103700008F7090E0029714F28091DA019091DB01C2
:103710009A838983BC82AB828091DE018D831E8275
:103720002F83CE010196B0CFA21AB30AF8ECAF16E0
:10373000B10408F042C0882309F447C0FE2CEE20F3
:1037400009F425CF8091DB018C1129C08091DA0129
:103750008D1125C09091E00190FD18C0892F8295B0
:103760008F70282F30E02115310581F0F801968304
:103770002F30310541F08F5F982F9295907F868191
:103780008F70892B8683C8010E940E0487E0F801A0
:10379000AAEDB1E001900D928A95E1F718C0C80139
:1037A0000E949024811172CF8091E001816080930A
:1037B000E001C8010E940E040AC087E0F4011192E2
:1037C0008A95E9F704C0F12C02C0FF24F3948F2DF1
:1037D0006496ECE00C941B2B9091B10121E030E059
:1037E000F90101C0EE0F8A95EAF7D90102C0AA0FCC
:1037F000BB1F6A95E2F7BD016E2B01C0220F4A95EF
:10380000EAF7892F8623681303C0892F822B03C010
:103810002095822F89230E947124089580910F01A1
:103820000895FC01EE0FFF1F8E0F9F1FFC01EC5847
:10383000FD4F6183408322830895249A089585B1C2
:103840008F7E95B190612FB7F894E4E7F2E032E013
:10385000EC38F30789F0319148E095B9000000C0D9
:1038600037FF85B9330F000000C000C000C085B924
:1038700000C04A9591F7EBCF2FBF8FE594E00197F9
:10388000F1F700C0000008950F931F93CF93DF93CB
:103890008B01EA019091D001943079F58F7080937B
:1038A000E9008FEF9091E800815095FD06C095EDFD
:1038B0009A95F1F700008111F5CF8091E80085FF1E
:1038C0001CC00E940516882361F08091E8008E7765
:1038D0008093E80012C0F80181918F018093F1007C
:1038E0002197209791F38091E80085FDF4CF809196
:1038F000E8008E778093E800E4CFDF91CF911F91AD
:103900000F91089540E250E0BC0184E00E94441C05
:103910000895CF93DF93EC0148E050E0BC0181E0D3
:103920000E94441C88E0FE01A6ECB1E001900D92DB
:103930008A95E1F7DF91CF91089587E797E7909314
:103940000108809300089AE088E10FB6F894A895E2
:10395000809360000FBE90936000FFCF78941F9219
:103960000F920FB60F9211248F939F93AF93BF9333
:103970008091A5029091A602A091A702B091A80201
:103980000196A11DB11D8093A5029093A602A0935C
:10399000A702B093A802BF91AF919F918F910F9012
:1039A0000FBE0F901F9018959C014FB7F89480910F
:1039B000A5029091A602A091A702B091A8024FBFC4
:1039C000821B930B08952FB7F8946091A502709114
:1039D000A6028091A7029091A8022FBF08952FB749
:1039E000F8948091A5029091A602A091A702B091AF
:1039F000A8022FBF08951F920F920FB60F921124A5
:103A00008F939F93AF93BF938091A402811113C0B2
:103A10008091A5029091A602A091A702B091A80260
:103A20004196A11DB11D8093A5029093A602A0937B
:103A3000A702B093A802BF91AF919F918F910F9071
:103A40000FBE0F901F90189590911001913021F4A6
:103A50009091A20297FD03C0ECE4F2E01DC0E82FB4
:103A6000E695E695E695EE31E0F4F0E0EC5AFD4F90
:103A7000877021E030E0A90102C0440F551F8A95EC
:103A8000E2F7CA0180959281892382830895319655
:103A900052E0E235F50729F092818913F8CF1282BE
:103AA000F6CF0895909110019130D1F49091A20237
:103AB00097FF16C0E82FE695E695E695EE3140F5BE
:103AC000F0E0EC5AFD4F877021E030E0A90102C020
:103AD000440F551F8A95E2F7CA019281892B16C0BF
:103AE000AEE4B2E0EFEF90E02D91821789F0EF3F66
:103AF00019F4211101C0E92F9F5F9630A9F7EF3F1C
:103B000039F00E2E000CFF0BE45BFD4F828308950D
:103B10000895A3E0B0E0EFE8FDE10C94092B2091BB
:103B2000A0023091A10228173907A1F09093A102B9
:103B30008093A002E0919E02F0919F02309751F095
:103B400024E029839B838A830084F185E02DCE01C4
:103B5000019609952396E2E00C94252BA3E0B0E0B2
:103B6000E4EBFDE10C94092B20919C0230919D0225
:103B700028173907A1F090939D0280939C02E09151
:103B80009E02F0919F02309751F023E029839B839E
:103B90008A830084F185E02DCE0101960995239654
:103BA000E2E00C94252BE0919E02F0919F02309769
:103BB00029F00190F081E02D0995089580E00895A5
:103BC00087E290E00E94022A0895CF93C82F8111C6
:103BD00002C06FEF01C065E284E290E00E94022A19
:103BE000C11102C06FEF01C061E085E290E00E9468
:103BF000022AC11102C06FEF01C064E186E290E0C9
:103C00000E94022ACF91089584E290E00E94DE296A
:103C1000853281F485E290E00E94DE29813051F402
:103C200086E290E00E94DE2991E0843109F090E084
:103C3000892F01C080E0817008950F931F93CF9367
:103C4000DF93C42FD22FFC0185818823B1F04093EC
:103C50009B020E94EF1C90939A028093990280E24B
:103C60008C0F883008F068C0C77081E001C0880FF1
:103C7000CA95EAF70E94EB245FC080919B0248132B
:103C80003DC08091990290919A020E94D41C883C78
:103C90009105A0F510E21D0FCD17E9F080E28C0F21
:103CA000883040F4C77081E001C0880FCA95EAF7F8
:103CB0000E94E424183078F581E09D2F977001C0B0
:103CC000880F9A95EAF70E94EB24093351F560E5D5
:103CD00070E089E329C0093319F460E570E002C09F
:103CE00060E070E0802F0E94DE26183028F5D77043
:103CF00081E001C0880FDA95EAF70AC080E28C0FF4
:103D00008830D0F4C77081E001C0880FCA95EAF707
:103D10000E94E42411C0093351F460E570E089E3A6
:103D200009C060E070E0802F0E94DE26E0CF60E0F6
:103D300070E0802F0E94DE26DF91CF911F910F91BE
:103D400008950E94EF1C20919502211104C020913A
:103D50009602222321F09093920280939102209167
:103D60009702211104C020919802222321F0909300
:103D7000900280938F02E0919E02F0919F02309713
:103D800049F082E0809393020680F781E02D83E979
:103D900092E00995089580918E0280FD16C081FD04
:103DA00016C082FD18C080918D02882391F0883260
:103DB00090F428E0829FC001112468E270E00E9424
:103DC000C92A862F672B29F007C082E0089584E076
:103DD000089581E0089588E0089580918E0280FD25
:103DE00014C081FD14C082FD16C080918C0288230E
:103DF00081F08E3180F420E5829FC00111246EE1B4
:103E000070E00E94C92A862F089584E1089588E20F
:103E1000089588E0089580E50895282F35EB230361
:103E2000C001112497FF03C08058910902C0805837
:103E30009F4F892F0895CF93DF93C8E2D2E060E0CF
:103E4000CE010E94022A2196C11584E0D807B9F755
:103E5000DF91CF9108951F93CF93DF93962F8430F6
:103E6000E8F46830D8F44830C8F4632F122FC42F18
:103E7000D0E0CC0FDD1F20E1929FC00DD11D112499
